S01800006275696C642F6D696361322F6D61696E2E737265632D
S11300000C9446000C9463000C9463000C946300FD
S11300100C9463000C9463000C9463000C946300D0
S11300200C9463000C9463000C9463000C946300C0
S11300300C9463000C9463000C9463000C9407010B
S11300400C9463000C9463000C9463000C946300A0
S11300500C9463000C9463000C9463000C94630090
S11300600C9463000C9463000C9463000C94630080
S11300700C9463000C9463000C9463000C94630070
S11300800C9463000C9463000C94630011241FBE51
S1130090CFEFD0E1DEBFCDBF11E0A0E0B1E0E8E9F1
S11300A0F2E000E00BBF02C007900D92A030B10750
S11300B0D9F711E0A0E0B1E001C01D92A831B10769
S11300C0E1F70C9494000C940000AC0180E00FB6AE
S11300D007FC81E0F894282F3327E09115018091E3
S11300E015018F5F809315018091150187708093AE
S11300F015019091150180911301981769F022233D
S113010009F07894FF27EE0FFF1FEE5FFE4F408348
S1130110518381E090E00895E0931501222309F0D2
S1130120789480E090E00895CFEFD0E1DEBFCDBFBA
S1130130D29AD09AD19AD698A79AA69AA59AA49A0E
S1130140A39AA29AA19AA09A8C9A8F9A8E9ABB98F3
S1130150BF98D39A8B9A8D9ADB9ADA9AD89AD99ABD
S113016083E08C5F8739E8F320E08AE08093000124
S113017020931501209313018FB7F89499272093A6
S11301801701DA9AD89AD99A8FBF9FE08FB7F8945B
S1130190482F552787B78E7F87BF87B78D7F87BF47
S11301A080B7886080BF93BF22BF91BF87B782604A
S11301B087BF4FBF789490911301809115019817D0
S11301C019F480E090E01AC090911301809113011A
S11301D08F5F8093130180911301877080931301C3
S11301E0E92FFF27EE0FFF1FEE5FFE4F8081918105
S11301F010821182FC01099581E090E08823D9F6F0
S113020085B7806285BF889500000000D4CF7894BC
S11302101F920F920FB60F9211242F933F938F9337
S11302209F938FB7F894282F332780910101882357
S113023069F0809114018093160188608093140101
S113024083BF8091120181BF109201012FBF8FB72C
S1130250F894382F2091170120FF06C08FB7F89427
S11302609927DA9A2E7F05C08FB7F8949927DA98E0
S11302702160209317018FBF3FBF9F918F913F91C2
S11302802F910F900FBE0F901F9018958FB7F89471
S10B0290992708958FBF08951A
S9030000FC
